:020000040000FA
:040000001C20462852
:08000800F300030EF400831263
:10001000031383130408F5000A08F6008A018C18FC
:1000200052208C1AF22376088A0075088400740E18
:100030008300F30E730E0900830103018500F100B4
:100040008600F2008316E0308500063086008312B9
:1000500083169630810083120C3097000030950093
:100060008316FF30920083120430920007309F0005
:10007000243083169800903083129800273083161E
:1000800099008C16831281018B010800A721ED20B5
:1000900083168C1483120B178B17C82103184D2855
:0400A000F0204D28D7
:0C00A4008C10F701F801831620102508CD
:1000B000A10726080318260FA20727080318270FF1
:1000C000A30728080318280FA407A01C79282408D0
:1000D0009B001C141A08FA00F9017A0DFA0CF90CAD
:1000E0007A0DFA0CF90C7908F7077A0803187A0FD9
:1000F000F80731103608B20737080318370FB3076F
:1001000038080318380FB40739080318390FB50732
:10011000B11C9C2835089B001C141A08FA00F90130
:100120007A0DFA0CF90C7A0DFA0CF90C7908F7072C
:100130007A0803187A0FF80742104708C3074808DF
:100140000318480FC40749080318490FC5074A0890
:1001500003184A0FC607C21CBF2846089B001C1480
:100160001A08FA00F9017A0DFA0CF90C7A0DFA0C5A
:10017000F90C7908F7077A0803187A0FF807531073
:100180005808D40759080318590FD5075A080318F7
:100190005A0FD6075B0803185B0FD707D31CE2285A
:1001A00057089B001C141A08FA00F9017A0DFA0C82
:1001B000F90C7A0DFA0CF90C7908F7077A0803188C
:1001C0007A0FF80783127808803E95009F309705D4
:0A01D000F71B1716771B971608009F
:0601DA00B3012F101229F1
:1001E000B000B01FFF28F8303002031808002F10AD
:1001F0003008B300F03030020318B30108002F1CA0
:100200000429B5002F104B29B30803190800B400C6
:10021000C0303302031C1029E0303302031C4B2989
:100220002F140800A030A900B130AA00C230AB00E2
:10023000D330AC00B0012930300784000008B20090
:1002400084008001840A8001840A8001840A80017C
:10025000840A8001840A8001840A8001840A800162
:10026000840A8001840AFF308000840A1F308000E5
:10027000840A3C308000840A8001840A8001840A58
:1002800002308000840A7F308000840A8000B00A37
:10029000301D1B2908000F303305B600043036022C
:1002A000031808003608293E84000008B600023012
:1002B0008A00330E0739F03E820002308A0034088B
:0C02C000003E8200B508031DF82A0D2B3B
:0402CC002008FC39D1
:1002D000A6002108A700A8010C30A702031C722960
:1002E000A80A6D29A7070030A6070318A70A04303B
:1002F000A707A3218A01A200A60AA3218A01A300BD
:10030000A60AA3218A01A400A60AA3218A01A500A6
:10031000A80E280E0A3C031C0301A800A81D98295A
:100320002308A2002408A3002508A400A501A81101
:10033000A8080319A2290310A50CA40CA30CA20C55
:0E034000A80B9B29080027088A0026088200C7
:02034E00031793
:100350008317E0012030E200E1000313831308005B
:1003600003178317E300601BC42962088400630835
:100370008000E00AE20A60306202031DC1292030D9
:10038000E20003138313080003138313701408009F
:1003900003178317E0080319DE29610884000008A9
:1003A000E400E003E10A60306102031DD929203036
:1003B000E10064080313831303100800031383137D
:0403C000031408001A
:10040000080008000800080008000800802A08000A
:10041000080008000800080008000800080008009C
:10042000080008000800080008000800080008008C
:10043000080008000800080008000800080008007C
:10044000080008000800080008000800080008006C
:10045000080008000800080008000800080008005C
:10046000080008000800080008000800080008004C
:10047000080008000800080008000800080008003C
:10048000080008000800080008000800080008002C
:10049000080008000800080008000800080008001C
:1004A000080008000800080008000800080008000C
:1004B00008000800080008000800080008000800FC
:1004C000922AA22AB12AB12AB92ABF2A0800080012
:1004D00008000800080008000800080008000800DC
:1004E00008000800080008000800080008000800CC
:1004F000202B392B202B202B202B202B202B202B8B
:1005000036080F3E84000008840A0004031D08001A
:100510000D3035020318080036080E3E84003508F9
:100520008000080036080F3E84000008840A00049A
:10053000031D080036080E3E84000C300002031D27
:10054000800A080036080F3E84000008840A000470
:10055000031D080036080E3E84000008031D8003BA
:10056000080036080F3E84007F308000840A800037
:10057000080036080F3E8400350880000800360861
:0A058000103E8400350880000800DA
:1005E0000D2B622908005D2908000800512B080026
:1005F00036080B3E8400340880009A233608093EF2
:1006000084003B0880003C08840A80003608003ED5
:100610008400801400148B17080036080B3E8400F9
:1006200034080002031D08003608003E8400801CC8
:1006300008000018192B8B13801000148B1708006A
:1006400036080E3E840002308000013084077F307F
:100650008000840A800036080C3E84008001840AF1
:1006600080019A233608003E8400801000148B1706
:10067000080036080E3E84000230800001308407F6
:100680007F308000840A800036080C3E84008001A0
:10069000840A80019A233608003E840000148B17D8
:1006A000080036080E3E84000008652336080C3E1C
:1006B000840039088000840A3A0880009A233608AA
:1006C000003E840000148B170800B901BA01B00085
:1006D00030080319992B0310B00D0310B40D03104B
:1006E000B40DB50D8030B5073508B100B11F802BB2
:1006F0003408B401B4023508B501031CB50FB502C6
:100700000830B200B00C031C8B2B3408B907350835
:100710000318350FBA07BA0CB90CB20B822BB11FF4
:10072000992B3908B901B9023A08BA01031CBA0F6A
:10073000BA02080036080B3E84000008A10002300F
:1007400084070008A107A11FAC2B0C30801FAA2B27
:10075000A102A32BA107A32B84030008A0006621FC
:100760003608003E84000018B32B3608053E84008E
:100770008B1322088000840A23088000840A24083E
:0A0780008000840A250880000800AC
:0407E00000340034AD
:0C07E40070101819F92B9818FC2B1A083B
:1007F000B0291A087014FF2B18121816701408006C
:10080000C734D434BB346D344C343234D5346D34C5
:10081000AF349534EE346D34F034FE3407346E3436
:1008200010346E3421346E341234E3343A346E347E
:10083000F5345D3454346E34BD34DE346D346E348E
:100840006A34653487346E34FE34F134A0346E3447
:1008500079348434BA346E34DD341C34D4346E3498
:100860002C34BB34ED346E3468345F3407346F3469
:100870009034093421346F34A734B9343A346F34A6
:10088000AE346F3454346F34A7342B346E346F3439
:100890009334ED3487346F347234B534A1346F340B
:1008A00048348334BB346F3414345734D5346F3404
:1008B000D9343034EF346F34973410340934703411
:1008C0005034F634223470340634E2343C3470341C
:1008D000BA34D334563470346D34CB34703470340D
:1008E0002134C9348A347034D734CC34A4347034CD
:1008F0009034D634BE3470344E34E634D834703448
:100900001234FC34F2347034DD3417340D34713465
:10091000B234393427347134913461344134713410
:100920007C348F345B3471347434C3347534713433
:100930007B34FD348F34713491343D34AA347134B6
:10094000B9348334C4347134F434CF34DE34713484
:1009500043342234F9347134A7347A341334723482
:100960002334D9342D347234B7343D34483472349E
:100970006434A834623472342D3419347D347234C2
:10098000133490349734723416340D34B2347234D4
:1009900039349034CC3472347D341934E7347234C1
:1009A000E334A834013473346D343E341C3473346E
:1009B0001C34DA3436347334F1347B3451347334C8
:1009C000EF3423346C3473341634D23486347334B5
:1009D00067348634A1347334E5344034BC34733422
:1009E00091340134D73473346C34C834F1347334F3
:1009F000773495340C347434B43468342734743414
:100A00002434423442347434CA3421345D3474346E
:100A1000A534073478347434B934F33492347434EC
:100A20000534E634AD3474348C34DE34C834743474
:100A30004F34DD34E33474345034E234FE347434EF
:100A40008F34ED34193475340F34FF343434753445
:100A5000D034163450347534D53434346B34753462
:100A60001E34593486347534AD348334A13475342E
:100A70008434B434BC347534A534EB34D734753491
:100A80000F342934F3347534C5346C340E34763471
:100A9000C934B634293476341C34073445347634BA
:100AA000BF345D3460347634B434BA347B34763455
:100AB000FC341D349734763498348734B234763429
:100AC0008B34F734CD347634D5346D34E934763420
:100AD0007934EA340434773477346D34203477341D
:100AE000D134F6343B347734883486345734773411
:100AF0009F341C34733477341634B9348E347734DD
:100B0000EE345B34AA3477342B340534C63477346E
:100B1000CC34B434E1347734D3346A34FD347734AC
:100B200042342734193478341A34EA34343478347B
:100B30005E34B334503478340D3483346C347834C8
:100B40002A34593488347834B7343534A43478347A
:100B5000B4341834C034783423340234DC34783478
:100B60000634F234F73478345E34E83413347934AC
:100B70002D34E5342F3479347434E8344B347934FB
:100B80003534F2346734793471340234843479344E
:100B900029341934A034793460343634BC3479348F
:100BA00016345A34D83479344E348434F4347934A5
:100BB0000834B53410347A344634EC342C347A3476
:100BC0000A342A3449347A3456346E3465347A34EB
:100BD0002A34B93481347A3488340A349E347A34ED
:100BE00072346234BA347A34E934C034D6347A3464
:100BF000EE342534F3347A34843491340F347B3436
:100C0000AC3403342C347B3467347C3448347B3448
:100C1000B734FB3464347B349E34813481347B3488
:100C20001C340E349E347B343334A134BA347B34D8
:100C3000E6343A34D7347B343534DB34F3347B3424
:100C40002134823410347C34AE342F342D347C344F
:100C5000DB34E33449347C34AB349E3466347C3446
:100C60001F34603483347C3438342834A0347C34EA
:100C7000F934F634BC347C346334CC34D9347C3429
:100C80007634A834F6347C3436348B3413347D34E3
:100C9000A334743430347D34BE3464344D347D3404
:100CA0008A345B346A347D340934593487347D3472
:100CB0003A345D34A4347D3421346834C1347D3415
:100CC000BE347934DE347D3413349234FB347D34D5
:100CD0002234B13418347E34ED34D63435347E3495
:100CE0007434033453347E34B934363470347E343F
:100CF000BF3470348D347E348634B134AA347E34BB
:100D00001034F934C7347E345E344734E5347E34ED
:100D100073349C3402347F345034F8341F347F34BD
:100D2000F5345A343D347F346634C4345A347F3415
:100D3000A334343478347F34AF34AB3495347F34D7
:100D400089342934B3347F343534AE34D0347F34ED
:100D5000B4343934EE347F340734CC340B3480343B
:100D600030346534293480343134053447348034A8
:100D70000A34AC3464348034BE3459348234803420
:100D80004F340E34A0348034BD34C934BD34803483
:100D90000B348C34DB34803439345534F9348034BA
:100DA0004B342534173481344034FC3434348134AA
:100DB0001B34DA3452348134DE34BE34703481343E
:100DC0008934AA348E3481341F349D34AC34813458
:100DD000A2349634CA34813412349734E8348134DE
:100DE00071349E3406348234C134AC3424348234B9
:100DF0000434C234423482343B34DE3460348234CE
:100E0000683401347F3482348C342B349D34823402
:100E1000A9345C34BB348234C1349434D934823440
:100E2000D534D334F7348234E73419341634833468
:100E3000F8346634343483340B34BB345234833462
:100E40002034163471348334393478348F34833415
:100E50005934E134AD34833480345134CC34833468
:100E6000B034C834EA348334EB344634093484343F
:100E70003234CC3427348434873458344634843480
:100E8000EC34EB3464348434633486348334843413
:100E9000EC342734A23484348A34D034C0348434DB
:100EA0003E348034DF3484340B343734FE348434BD
:100EB000F034F4341C348534F134B9343B348534A3
:100EC0000E3486345A3485344A345934793485346E
:100ED000A63433349834853424341534B734853407
:100EE000C534FD34D53485348C34ED34F434853454
:100EF0007934E434133486348E34E2343234863434
:100F0000CD34E734513486343834F4347034863494
:100F1000D03407349034863497342234AF34863456
:100F20008F344434CE348634B9346D34ED34863461
:100F300017349E340C348734AB34D5342B34873497
:100F4000763414344B34873479345A346A348734E1
:100F5000B834A734893487343334FC34A834873424
:100F6000EB345734C8348734E434BA34E734873444
:100F70001D342534073488349A3496342634883422
:100F80005B340F344634883463348F3465348834AA
:100F9000B3341634853488344C34A534A4348834BE
:100FA00031343B34C43488346334D834E334883443
:100FB000E3347C3403348934B4342834233489341E
:100FC000D734DB34423489344F3496346234893434
:100FD0001B345834823489343F342134A234893468
:100FE000BC34F134C13489349334C934E1348934A4
:100FF000C734A83401348A3459348F3421348A34C4
:101000004A347D3441348A349D34723461348A34B4
:1010100053346F3481348A346E347334A1348A3457
:10102000EF347E34C1348A34D9349134E1348A3493
:101030002D34AC3401348B34EC34CD3421348B3446
:101040001934F73441348B34B534273462348B345B
:10105000C2345F3482348B3441349F34A2348B34B5
:101060003534E634C2348B349E343434E3348B3438
:1010700080348A3403348C34DB34E73423348C34C6
:10108000B1344C3444348C340434B93464348C3446
:10109000D5342C3485348C342734A834A5348C349E
:1010A000FB342A34C6348C345334B534E6348C34AF
:1010B0003134473407348D349634E03427348D345A
:1010C0008334813448348D34FC34293469348D348C
:1010D0000134DA3489348D3495349134AA348D3422
:1010E000B9345034CB348D346E341734EC348D3401
:1010F000B734E5340C348E349534BB342D348E340F
:101100000A3499344E348E3418347E346F348E342D
:10111000C1346A3490348E3406345F34B1348E3442
:10112000E9345A34D2348E346C345E34F3348E3431
:101130009034693414348F3458347C3435348F34DB
:10114000C534963456348F34D934B83477348F3428
:101150009534E23498348F34FC341334BA348F34F9
:101160000F344D34DB348F34D0348D34FC348F3431
:101170004134D6341D349034643426343F349034B2
:1011800039347E3460349034C434DD348134903466
:1011900006344534A33490340034B434C434903429
:1011A000B5342A34E63490342634A93407349134E3
:1011B00055342F34293491344334BD344A34913476
:1011C000F43452346C3491346734F0348D349134C7
:1011D000A0349534AF349134A0344234D1349134B6
:1011E0006934F734F2349134FC34B3341434923427
:1011F0005C347834363492348934443458349234FC
:10120000873418347A3492345734F4349B3492341B
:10121000FA34D734BD3492347234C334DF34923468
:10122000C234B63401349334EB34B13423349334C0
:10123000EF34B43445349334CF34BF34673493340B
:101240008E34D234893493342D34ED34AB3493342A
:10125000AE340F34CE34933413343A34F034933400
:101260005E346C34123494349034A6343434943470
:10127000AC34E83456349434B3343234793494345E
:10128000A73484349B3494348A34DE34BD349434AB
:101290005E344034E03494342434AA340234953437
:1012A000DF341B34253495349034953447349534E9
:1012B000393417346A349534DC34A0348C349534A2
:1012C0007B343234AF3495341834CC34D134953443
:1012D000B3346D34F43495345134173417349634B0
:1012E000F134C83439349634963482345C349634CC
:1012F000433444347F349634F8340D34A234963475
:10130000B734DF34C43496348334B934E734963494
:101310005E349B340A349734483485342D34973402
:1013200045347734503497345534713473349734AA
:101330007B34733496349734B9347D34B93497346C
:1013400010349034DC3497348334AA34FF34973427
:101350001334CD3422349834C234F73445349834BD
:1013600092342A3469349834853465348C34983412
:101370009D34A834AF349834DB34F334D234983409
:1013800042344734F6349834D334A234193499347F
:10139000913406343D3499347D3472346034993458
:1013A0009834E63483349934E6346234A73499347B
:1013B0006834E734CA3499341F347434EE349934C1
:1013C0000E34093412349A343734A63435349A340E
:1013D0009B344B3459349A343D34F9347C349A3448
:1013E0001D34AF34A0349A343F346D34C4349A344D
:1013F000A4343334E8349A344E3402340C349B34FD
:101400003F34D9342F349B347934B83453349B343B
:10141000FE349F3477349B34CF348F349B349B34E9
:10142000EE348734BF349B345F348834E3349B34E8
:101430002134913407349C343834A2342B349C3416
:10144000A534BB344F349C346B34DD3473349C345A
:101450008A34073498349C3406343A34BC349C348F
:10146000DF347434E0349C341934B83404349D349B
:10147000B434033429349D34B33457344D349D345B
:101480001834B43471349D34E434183496349D34B3
:101490001A348634BA349D34BC34FB34DE349D3483
:1014A000CB34793403349E344A34003428349E34A7
:1014B0003A348F344C349E349D34263471349E3407
:1014C0007634C63495349E34C5346E34BA349E3482
:1014D0008E341F34DF349E34D334D83403349F34F5
:1014E00094349A3428349F34D53464344D349F3442
:1014F0009634373472349F34DB34123497349F344B
:10150000A434F634BB349F34F534E234E0349F34F1
:10151000CE34D7340534A0343334D5342A34A0340F
:101520002434DB344F34A034A434E9347434A0348C
:10153000B53400349A34A03459342034BF34A03444
:1015400091344834E434A034613479340934A1341A
:10155000C934B2342E34A134CC34F4345334A134ED
:101560006B343F347934A134AA3492349E34A1349C
:101570008934EE34C334A1340B345334E934A13408
:101580003134C0340E34A234FE3435343434A23411
:101590007434B4345934A23495343B347F34A23497
:1015A0006234CB34A434A234DF346334CA34A2347A
:1015B0000B340534F034A234EB34AE341534A33498
:1015C0007F3461343B34A334CA341C346134A334D3
:1015D000CE34E0348634A3348D34AD34AC34A3340B
:1015E00008348334D234A33443346134F834A3341C
:1015F0003E3448341E34A434FC3437344434A434E8
:101600007F3430346A34A434C93431349034A4344F
:10161000DC343B34B634A434B9344E34DC34A43432
:1016200064346A340234A534DE348E342834A5346C
:101630002934BC344E34A5344734F2347434A534E0
:101640003A3431349B34A53405347934C134A5346B
:10165000A934C934E734A534283423340E34A634ED
:10166000843485343434A634C034F0345A34A63447
:10167000DD3464348134A634DE34E134A734A63456
:10168000C4346734CE34A6349234F634F434A634F9
:101690004A348E341B34A734ED342E344234A7340C
:1016A0007E34D8346834A734FF348A348F34A73476
:1016B00072344634B634A734D9340A34DD34A7340E
:1016C0003634D8340334A8348B34AE342A34A834B6
:1016D000DA348D345134A834263476347834A8344E
:1016E000703467349F34A834BA346134C634A834B3
:1016F00007346534ED34A834583471341434A934C3
:10170000B03486343B34A9341134A5346234A9345E
:101710007D34CC348934A934F634FC34B034A93463
:101720007D343634D834A93416347934FF34A934AE
:10173000C234C4342634AA34843419344E34AA341E
:101740005D3477347534AA344F34DE349C34AA3493
:101750005D344E34C434AA348934C734EB34AA34EB
:10176000D43449341334AB344234D5343A34AB3402
:10177000D33469346234AB348B3407348A34AB34B9
:101780006B34AE34B134AB3476345E34D934AB34EC
:10179000AD3417340134AC341234DA342834AC3478
:1017A000A934A5345034AC3472347A347834AC343F
:1017B00071345834A034AC34A6343F34C834AC341B
:1017C00015343034F034AC34BF3429341834AD34EB
:1017D000A7342C344034AD34CE3438346834AD348E
:1017E00037344E349034AD34E5346C34B834AD34E1
:1017F000D8349434E034AD341434C6340834AE34C0
:10180000993400343134AE346C3444345934AE3409
:101810008D3491348134AE34FF34E734A934AE349E
:10182000C4344734D234AE34DE34B034FA34AE3457
:10183000503423342334AF341B349F344B34AF340F
:10184000413424347434AF34C534B2349C34AF34AE
:10185000AA344A34C534AF34F034EB34ED34AF3409
:101860009B3496341634B034AC344A343F34B034FC
:10187000263408346834B0340A34CF349034B03469
:101880005C349F34B934B0341D347934E234B0342C
:101890004F345C340B34B134F43448343434B13420
:1018A00010343F345D34B134A3343E348634B13423
:1018B000B0344734AF34B1343A345A34D834B13414
:1018C000423476340134B234CB349B342A34B234CB
:1018D000D634CA345334B234673403347D34B2342A
:1018E0007F344534A634B23420349134CF34B2340A
:1018F0004D34E634F834B234083445342234B33449
:101900005334AD344B34B33430341F347534B334C2
:10191000A2349A349E34B334AB341F34C834B33455
:101920004C34AE34F134B334893446341B34B434DB
:101930006334E8344434B434DC3493346E34B43433
:10194000F83448349834B434B7340734C234B43437
:101950001D34D034EB34B4342B34A2341534B534C4
:10196000E4347D343F34B5344A3463346934B534B7
:101970005F3452349334B53426344B34BD34B534EB
:10198000A0344D34E734B534D03459341134B6343E
:10199000B9346F343B34B6345C348F346534B63488
:1019A000BB34B8348F34B634DA34EB34B934B634AB
:1019B000B9342834E434B6345C346F340E34B7347C
:1019C000C534BF343834B734F63419346334B734DB
:1019D000F1347D348D34B734B834EB34B734B734A4
:1019E0004E346334E234B734B534E4340C34B834B0
:1019F000F0346F343734B834003405346234B834DA
:101A0000E734A3348C34B834A9344C34B734B83404
:101A10004734FF34E134B834C434BB340C34B93403
:101A2000223482343734B934633452346234B934B2
:101A300089342C348D34B93498341034B834B934F2
:101A40009034FE34E234B9347534F6340D34BA349B
:101A50004834F8343834BA340D3404346434BA3485
:101A6000C43419348F34BA3471343934BA34BA3492
:101A700016346334E534BA34B63496341034BB3497
:101A80005134D4343B34BB34EC341B346734BB3472
:101A900087346D349234BB342634C934BD34BB34FE
:101AA000CB342E34E934BB3477349E341434BC3414
:101AB0002E3418344034BC34F2349B346B34BC3490
:101AC000C53429349734BC34A934C134C234BC344D
:101AD000A0346334EE34BC34AE340F341A34BD3425
:101AE000D434C5344534BD34153486347134BD34F2
:101AF000723450349D34BD34EF342434C934BD3491
:101B00008D340334F534BD345034EC342034BE34D9
:101B10003934DF344C34BE344A34DC347834BE34A7
:101B20008734E334A434BE34F134F434D034BE34D6
:101B30008B341034FD34BE34563436342934BF343B
:101B4000573466345534BF348E34A0348134BF34B6
:101B5000FE34E434AD34BF34A9343334DA34BF3422
:101B600093348C340634C034BD34EF343234C03452
:101B70002A345D345F34C034DB34D4348B34C03425
:101B8000D4345634B834C0341734E334E434C03475
:101B9000A53479341134C13483341A343E34C13419
:101BA000B134C5346A34C13432347B349734C134EF
:101BB0000A343B34C434C13439340534F134C134CB
:101BC000C234D9341D34C234A934B8344A34C2348E
:101BD000EF34A1347734C23496349534A434C2340B
:101BE000A1349334D134C23413349C34FE34C2341F
:101BF000EE34AE342B34C3343434CC345834C334A0
:101C0000E734F3348534C3340B342634B334C3346B
:101C1000A1346234E034C334AC34A9340D34C43458
:101C20002E34FB343A34C4342B3457346834C4343F
:101C3000A334BD349534C43499342E34C334C434FD
:101C40001134AA34F034C4340C3430341E34C53466
:101C50008D34C0344B34C53497345B347934C53457
:101C60002B340134A734C5344C34B134D434C534A6
:101C7000FD346B340234C634403431343034C6342D
:101C8000173401345E34C6348534DB348B34C634C7
:101C90008D34C034B934C6343034B034E734C6344B
:101CA0007234AA341534C7345534AF344334C7348E
:101CB000DA34BE347134C7340634D9349F34C7346F
:101CC000D934FD34CD34C73457342D34FC34C734C3
:101CD000823467342A34C8345D34AC345834C83460
:101CE000E934FB348634C8342A345634B534C83425
:101CF0002234BB34E334C834D4342A341234C934E3
:101D00004134A5344034C9346C342A346F34C93476
:101D10005934BA349D34C93408345534CC34C934B8
:101D20007E34FA34FA34C934BC34AA342934CA347F
:101D3000C43465345834CA349A342B348734CA34A2
:101D40004034FC34B534CA34B834D734E434CA34FB
:101D50000534BE341334CB342934AF344234CB345D
:101D60002734AB347134CB340134B234A034CB34A7
:101D7000BA34C334CF34CB345534E034FE34CB34AE
:101D8000D33407342E34CC3438343A345D34CC3444
:101D9000853477348C34CC34BE34BF34BB34CC344B
:101DA000E5341234EB34CC34FC3470341A34CD3492
:101DB0000634DA344934CD3406344E347934CD34F3
:101DC000FE34CC34A834CD34F1345634D834CD3448
:101DD000E034EB340734CE34CF348B343734CE3464
:101DE000C13436346734CE34B734EC349634CE3420
:101DF000B434AD34C634CE34BC347934F634CE3455
:101E0000CF3450342634CF34F23432345634CF34D5
:101E1000263420348634CF346F341834B634CF347B
:101E2000CD341B34E634CF3446342A341634D0341F
:101E3000D93443344634D0348C3468347634D03496
:101E40005F349834A634D0345534D334D634D034B7
:101E5000723419340734D134B7346A343734D13456
:101E60002734C7346734D134C5342E349834D13450
:101E70009434A134C834D13495341F34F934D13476
:101E8000CC34A8342934D2343C343D345A34D2349E
:101E9000E534DC348A34D234CD348734BB34D234A4
:101EA000F4343D34EC34D2345D34FF341C34D33458
:101EB0000C34CC344D34D3340334A4347E34D33492
:101EC00043348734AF34D334D1347534E034D3342D
:101ED000AE346F341134D434DE3474344234D434F8
:101EE000623485347334D4343E34A134A434D434CD
:101EF0007334C834D534D4340634FB340634D53482
:101F0000F73438343834D5344B3482346934D534EA
:101F10000334D7349A34D53422343734CC34D534DE
:101F2000AB34A234FD34D534A13419342F34D63433
:101F300005349C346034D634DC3429349234D634BD
:101F40002634C334C334D634E8346734F534D63455
:101F5000233418342734D734DB34D3345834D734CB
:101F600012349B348A34D734CA346D34BC34D734F9
:101F700007344C34EE34D734CA3435342034D834B2
:101F800017342B345234D834F1342B348434D834CD
:101F900059343834B634D83453345034E834D8341F
:101FA000E23473341A34D9340734A3344C34D9347A
:101FB000C634DD347E34D93421342434B134D934B8
:101FC0001C347634E334D934B834D3341534DA34A9
:101FD000F8343C344834DA34E034B1347A34DA3426
:101FE00071343234AD34DA34AF34BE34DF34DA3401
:101FF0009C3456341234DB343B34FA344434DB340E
:084000000000050000000100B2
:02400E00623F0F
:10420000000007000F0017001F0026002E003500D9
:104210003C00430049004F0054005A005F00630017
:1042200067006B006E007100740076007800790002
:104230007A007B007C007C007C007C007C007B00A2
:104240007B007A007A0079007800780077007700A8
:1042500076007600750075007500750075007500B4
:1042600076007600770077007800790079007A0090
:104270007B007C007C007D007D007E007E007E0057
:104280007E007E007E007E007D007C007C007A0047
:104290007900780076007400720070006E006B0088
:1042A00069006600630060005D005A00570054001A
:1042B00051004E004B0049004600430040003D00C5
:1042C0003B0038003500330031002E002C002A005E
:1042D000280026002400220020001F001D001B00D3
:1042E00019001800160015001300110010000E0030
:1042F0000D000B0009000800060004000300010087
:104300000000FF00FD00FC00FA00F800F700F500D7
:10431000F300F200F000EF00ED00EB00EA00E8002F
:10432000E700E500E300E100E000DE00DC00DA0089
:10433000D800D600D400D200CF00CD00CB00C800FA
:10434000C500C300C000BD00BA00B700B500B20090
:10435000AF00AC00A900A600A300A0009D009A0039
:1043600097009500920090008E008C008A008800D3
:10437000870086008400840083008200820082001F
:104380008200820082008200830083008400840017
:1043900085008600870087008800890089008A00E0
:1043A0008A008B008B008B008B008B008B008A00B7
:1043B0008A008900890088008800870086008600BE
:1043C00085008500840084008400840084008500CA
:1043D0008600870088008A008C008F00920095007C
:1043E00099009D00A100A600AC00B100B700BD007F
:1043F000C400CB00D200DA00E100E900F100F900CE
:00000001FF
